:0200000480007A
:100000006F008004732F2034930F80006308FF0378
:10001000930F90006304FF03930FB0006300FF038E
:10002000130F000063040F0067000F00732F2034CC
:1000300063540F006F00400093E19153171F0000BD
:1000400023223FFC6FF09FFF93000000130100008C
:10005000930100001302000093020000130300004C
:100060009303000013040000930400001305000034
:10007000930500001306000093060000130700001C
:100080009307000013080000930800001309000004
:1000900093090000130A0000930A0000130B0000EC
:1000A000930B0000130C0000930C0000130D0000D4
:1000B000930D0000130E0000930E0000130F0000BC
:1000C000930F0000732540F16310050097020000B4
:1000D000938202017390523073500018970200000F
:1000E00093824202739052309B021000939252030B
:1000F0009382F2FF7390023B9302F0017390023AF5
:100100007350403097020000938242017390523046
:10011000735020307350303093010000970200007C
:10012000938282EE73905230130510001315F5017F
:10013000635C05000F00F00F930110009308D005D9
:10014000130500007300000093020000638A0200A0
:1001500073905210B7B200009B82921073902230BD
:100160007350003097020000938242017390123462
:10017000732540F173002030930010001B9700009E
:100180009303100093012000631277309300100056
:100190001B97100093032000930130006318772E03
:1001A000930010001B977000930300089301400018
:1001B000631E772C930010001B97E000B7430000EC
:1001C000930150006314772C930010001B97F001EB
:1001D000B703008093016000631A772A9300F0FF51
:1001E0001B9700009303F0FF930170006310772AC0
:1001F0009300F0FF1B9710009303E0FF9301800032
:10020000631677289300F0FF1B977000930300F8A4
:1002100093019000631C77269300F0FF1B97E0008A
:10022000B7C3FFFF9301A000631277269300F0FF8E
:100230001B97F001B70300809301B0006318772487
:10024000B72021219B8010121B970000B72321218A
:100250009B8313129301C000631A7722B7202121D8
:100260009B8010121B971000B74342429B832324AC
:100270009301D000631C7720B72021219B801012AE
:100280001B977000B79390909B8303089301E00045
:10029000631E771EB72021219B8010121B97E00060
:1002A000B74348489301F0006312771EB72021211D
:1002B0009B8010121B97F001B7030080930100018F
:1002C0006316771CB720F1FF9B8050349390C000D9
:1002D000938080671B970000B75334129B8383671A
:1002E0009301C0026314771AB720F1FF9B8050344A
:1002F0009390C000938080671B974000B7634523AD
:100300009B8303789301D00263127718B72009000A
:100310009B8050349390C000938080671B970000AF
:10032000B75334929B8383679301E002631077167F
:10033000B79009009B8050349390C00093808067F1
:100340001B974000B76345939B8303789301F002AA
:10035000631E7712930010009B90700093030008B7
:1003600093011001639470121302000093001000B7
:100370001B97700013030700130212009302200062
:10038000E31652FE930300089301200163107310DB
:1003900013020000930010001B97E0001300000000
:1003A000130307001302120093022000E31452FE0D
:1003B000B743000093013001631A730C130200006D
:1003C000930010001B97F0011300000013000000C1
:1003D000130307001302120093022000E31252FEDF
:1003E000B7030080930140016312730A13020000F7
:1003F000930010001B97700013021200930220005C
:10040000E31852FE9303000893015001631077082C
:100410001302000093001000130000001B97E0007F
:100420001302120093022000E31652FEB7430000AD
:1004300093016001631C7704130200009300100015
:1004400013000000130000001B97F00113021200BC
:1004500093022000E31452FEB70300809301700161
:10046000631677029B10F001930300009301800153
:10047000639E70009300F0011B90C0019303000085
:100480009301900163147000631030020F00F00FAD
:10049000638001009391110093E111009308D0054E
:1004A00013850100730000000F00F00F930110008E
:1004B0009308D0051305000073000000731000C0FE
:1004C000000000000000000000000000000000002C
:1004D000000000000000000000000000000000001C
:1004E000000000000000000000000000000000000C
:0C04F00000000000000000000000000000
:1010000000000000000000000000000000000000E0
:1010100000000000000000000000000000000000D0
:1010200000000000000000000000000000000000C0
:1010300000000000000000000000000000000000B0
:081040000000000000000000A8
:040000058000000077
:00000001FF
